:100000001DC037C036C014C134C033C032C031C087
:1000100067C12FC02EC02DC02CC02BC02AC000002D
:100020000000370000000000380002020202020255
:1000300001020408102001030000040011241FBE67
:10004000CFE5D2E0DEBFCDBF10E0A0E6B0E0E8EF44
:10005000F8E002C005900D92AA38B107D9F721E067
:10006000AAE8B0E001C01D92A53AB207E1F71FD29D
:1000700041C4C6CF17B8379A329A319A309A339A18
:100080008FB780688FBF089580919701982F990F3F
:100090009093970120919100309192003695279589
:1000A000369527952639310520F4881F8827881F23
:1000B00007C0233A3105D0F182B787FB882780F942
:1000C000882319F0916090939701109299011092F2
:1000D00098012091970120FF06C081E090E0909365
:1000E000990180939801809198019091990123FF43
:1000F0001FC082609093990180939801809198012C
:100100009091990125FF16C0846090939901809386
:100110009801E0919801F0919901EE57FF4F80818D
:1001200090E0909399018093980108958095BDCFB8
:100130008D7FE0CF8B7FE9CF90E0FC01EA5CFF4F41
:100140003491FC01E05DFF4F2491FC01E65DFF4F1F
:10015000E491EE23B9F0332329F03130A1F48AB5CC
:100160008F778ABDF0E0EE0FFF1FEC5DFF4FA5918A
:10017000B4918FB7611118C0F894EC9120952E239B
:100180002C938FBF0895323019F48AB58F7DE9CF53
:10019000333021F480B78F7D80BFE4CF343011F746
:1001A0008CB58F7D8CBDDECFF894EC912E2BE8CFF3
:1001B000CF93DF9387FF07C08F7769F1813069F1B3
:1001C000823069F183E090E0FC01E05DFF4F249113
:1001D000865D9F4FFC0184918823D1F090E0880FC9
:1001E000991FFC01E25EFF4FA591B491FC01EC5D0B
:1001F000FF4FC591D491611114C09FB7F8948C91B1
:10020000E22FE0958E238C932881E223E8839FBF21
:10021000DF91CF91089585E0D6CF82E0D4CF84E0FE
:10022000D2CF8FB7F894EC91E22BEC938FBFF0CF45
:100230001F920F920FB60F9211242F933F934F935B
:100240005F936F937F938F939F9380919D018F5FB7
:1002500080939D0181111FC09091750021E092272C
:10026000909375009923A9F140919F015091A001AD
:100270006091A1017091A2014530510561057105A0
:1002800028F110929E0110929F011092A0011092ED
:10029000A1011092A20190E0209175002223D9F0D3
:1002A0002FEF30E0281B390B30939B0120939A01EC
:1002B0001FBC9F918F917F916F915F914F913F9163
:1002C0002F910F900FBE0F901F90189520939E01B5
:1002D000DACF90E080E090939B0180939A01E8CF81
:1002E0001F920F920FB60F921124CF92DF92EF92CE
:1002F000FF922F933F934F935F936F937F938F93CF
:100300009F93AF93BF93EF93FF938091740090916D
:100310009000911197C0E82FF0E0EE0FFF1FDF0172
:10032000A657BF4FEF56FF4F208131812D933C934D
:1003300094B125B1322F292F31832083823009F0E7
:1003400047C0809195009091960020918E00309149
:100350008F0028173907E1F196958795969587952F
:10036000FC01E956FF4F208130E043E0220F331FAC
:100370004A95E1F784E198E0821B930BFC01EE0FB4
:10038000EF2FEE1FFF0BEF5F30E020E0C12CD12CF0
:100390007601C394F0E0B701A601022E04C0440F19
:1003A000551F661F771F0A94D2F7DF01022E02C085
:1003B000B595A7950A94E2F7A0FF19C0A0B74A2BFC
:1003C00040BF2F5F3F4F2430310529F780688EBD35
:1003D000909174009F5F892FE82FF0E0E258FF4F63
:1003E0009081911108C08F5F8430B0F3F4CFA0B733
:1003F00040954A23E5CF833018F5809374008091AF
:10040000740097B1907797B997B1892B87B981E03C
:1004100080939000369AFF91EF91BF91AF919F9199
:100420008F917F916F915F914F913F912F91FF90AD
:10043000EF90DF90CF900F900FBE0F901F90189508
:1004400082E0DBCF823081F580919500909196001B
:100450008E3E924008F4BC9A27B3E0917400F0E01D
:10046000E658FF4F308181E090E0A0E0B0E0AC01C1
:10047000BD0104C0440F551F661F771F3A95D2F780
:100480004095422347BB28B3E0917400F0E0E65862
:10049000FF4F308104C0880F991FAA1FBB1F3A95D8
:1004A000D2F78095822388BB10929000B3CFCF9370
:1004B000DF9300D000D000D0CDB7DEB7DBDD61E048
:1004C00085E03ADE60E084E073DE61E084E034DE03
:1004D00077E9272E70E0372EC12CD12C76018601CA
:1004E0002FEF30E040E050E0812C912C54016FEF71
:1004F00070E080E090E069837A838B839C83412C59
:10050000512C320190E080E0DC01AA0FBB1FFD01FD
:10051000E05AFF4F608171817E836D830617170754
:1005200018F1FD01EE59FF4F60817181601771076D
:10053000D8F09B0150E040E029833A834B835C83F1
:100540004D815E812A01712C612CFD01E459FF4F20
:100550002081318150E040E0A659BF4F8D909C90A2
:10056000B12CA12C8FE090E001968430910564F2CB
:10057000C701B6016419750986099709281939094F
:100580004A095B0960D129813A814B815C81241938
:1005900035094609570970D1820E931EA41EB51E57
:1005A000D1018D921D01BFEFCB1ADB0AEB0AFB0ACA
:1005B000C114E1E0DE06E104F10409F090CF83EA22
:1005C0008ABD81E083BF10BE1FBC82E08CBD8AEF74
:1005D0008EBD80E489BF84E880BF80B78B7F80BFF9
:1005E0007894DAD02FEF30E040E050E045D16093CE
:1005F000970161E080E0DCDD60E081E8D9DD60E06A
:1006000082E8D6DD60E083E8D3DD61E081E0D0DD23
:1006100061E082E0CDDD60E083E0CADD60E084E09F
:10062000C7DD60E084E088DD25DD8091740097B14E
:10063000907797B997B1892B87B9369A86B3F1E04D
:10064000F983982F987083FF198229812093A40140
:100650008091A301811124C0992311F180919F0100
:100660009091A001A091A101B091A2010196A11DBC
:10067000B11D80939F019093A001A093A101B0931D
:10068000A2010997A105B10510F010929E01809179
:100690009E01882321F010929D0110927500F4DCD8
:1006A00039813093A30180919C0190919D0197FD28
:1006B00021C041E040939C0150919C0159838517D2
:1006C00041F080919E018111DFDC69816623A9F0F0
:1006D000C29A80919A0190919B0197FD10C08F3F23
:1006E000910519F014F08FEF90E088BD809198018A
:1006F00089BDA4CF10929C01DFCFC298EACF80E0E1
:10070000F4CF8F929F92AF92BF92CF92DF92EF92EF
:10071000FF92CF93DF93EC01688179818A819B817D
:10072000611571058105910521F464E279ED8BE590
:1007300097E02DE133EF41E050E09ED049015A01AE
:1007400027EA31E440E050E07ED06B017C012CEEE2
:1007500034EF4FEF5FEFC501B40175D0C60ED71E61
:10076000E81EF91EF7FE06C081E0C81AD108E108AC
:1007700080E8F80AC882D982EA82FB82C701B60102
:100780009F77DF91CF91FF90EF90DF90CF90BF9058
:10079000AF909F908F9008958F929F92AF92BF924B
:1007A000CF92DF92EF92FF92609176007091770086
:1007B000809178009091790061157105810591050E
:1007C00021F464E279ED8BE597E02DE133EF41E030
:1007D00050E052D049015A0127EA31E440E050E0AC
:1007E00032D06B017C012CEE34EF4FEF5FEFC5018F
:1007F000B40129D0C60ED71EE81EF91EF7FE06C0AA
:1008000081E0C81AD108E10880E8F80AC0927600B1
:10081000D0927700E0927800F0927900C701B6019B
:100820009F77FF90EF90DF90CF90BF90AF909F9019
:100830008F9008956093760070937700809378008E
:10084000909379000895EE27FF27AA27BB2708C0B9
:10085000A20FB31FE41FF51F220F331F441F551FA4
:10086000969587957795679598F37040A9F70097C7
:1008700099F7BD01CF010895052E97FB16F400945A
:100880000FD057FD05D014D007FC02D046F408C0A5
:1008900050954095309521953F4F4F4F5F4F0895AC
:1008A00090958095709561957F4F8F4F9F4F0895DC
:1008B000A1E21A2EAA1BBB1BFD010DC0AA1FBB1F64
:1008C000EE1FFF1FA217B307E407F50720F0A21BD6
:1008D000B30BE40BF50B661F771F881F991F1A9443
:1008E00069F760957095809590959B01AC01BD016D
:0808F000CF010895F894FFCF39
:1008F800000032007F00BF00FF0050009D00B400E0
:10090800DC00FE00010101000000070204030100F1
:0A091800010000507896B4C8DCFF1F
:00000001FF
